:1000000089C300000C94D92EA2C30000A0C3000035
:100010009EC300009CC300009AC3000098C3000068
:1000200096C3000094C300000C940F2D0C94F72D80
:100030000C94C42C8CC300008AC3000088C3000049
:1000400086C3000084C3000082C3000080C3000098
:100050007EC300000C94EB2C7AC3000078C3000030
:1000600076C3000074C3000072C3000070C30000B8
:100070006EC300006CC300006AC3000068C30000C8
:1000800066C3000064C3000062C3000060C30000D8
:100090005EC300005CC300005AC3000058C30000E8
:1000A00056C3000054C3000052C3000005010902FA
:1000B000A10185020901A1000509190129081500FE
:1000C0002501950875018102050109300931158165
:1000D000257F95027508810609381581257F9501D0
:1000E00075088106050C0A38021581257F95017572
:1000F000088106C0C005010980A101850319012AF4
:10010000B700150126B700950175108100C0050CD8
:100110000901A101850419012AA002150126A002E6
:10012000950175108100C00660FF0961A101096297
:10013000150026FF00952075088102096315002629
:10014000FF00952075089102C005010906A101056F
:100150000719E029E7150025019508750181029529
:1001600001750881010507190029FF150026FF0008
:100170009506750881000508190129051500250156
:10018000950575019102950175039101C00000006C
:10019000000000000000000000000000000000005F
:1001A000000000000000000000000000000000004F
:1001B000007E0F00D4FFFFFFC700000078000000A2
:1001C00000000000002A2B280000000000000000B2
:1001D000000000000000000029000000002C1E3478
:1001E00020212224342627252E362D3738271E1F7E
:1001F000202122232425263333362E37381F0405A9
:10020000060708090A0B0C0D0E0F10111213141516
:10021000161718191A1B1C1D2F3130232D350405F4
:10022000060708090A0B0C0D0E0F101112131415F6
:10023000161718191A1B1C1D2F3130354C09025B7B
:1002400000030100A0FA09040000010301010009F4
:100250002111010001224400070581030800010962
:100260000401000203000000092111010001222203
:100270000007058203200001070503032000010990
:100280000402000103000000092111010001227B8A
:10029000000705840320000112010002000000088D
:1002A00010CB56110001010203011C037600690006
:1002B00061006C003A0066003600340063003200D2
:1002C00062003300630000001E034E0079007100DD
:1002D000750069007300740020005200650076000C
:1002E0002E002000310000000E034B006500650069
:1002F000620069006F0000000403090435001E005D
:100300001F002000210022002B0014001A0008000A
:1003100015001700290004001600070009000A0054
:10032000E1001D001B000600190005002552E00039
:10033000E200E30023522C002A00270026002500BB
:10034000240023004C00130012000C0018001C00B5
:10035000340033000F000E000D000B0028003800A1
:1003600037003600100011004F00520051005000BD
:1003700024522C0035001E001F0020002100220006
:100380002B0014001A00090013000A0029000400C1
:100390001500160017000700E1001D001B000600F5
:1003A000190005002552E000E200E30023522C0072
:1003B0002A00270026002500240023004C003300DB
:1003C0001C0018000F000D00340012000C00080083
:1003D00011000B00280038003700360010000E0016
:1003E0004F0052005100500024522C0035001E00D6
:1003F0001F002000210022002B00340036003700AF
:1004000013001C00290004001200080018000C0052
:10041000E100330014000D000E001B002552E00027
:10042000E200E30023522C002A00270026002500CA
:10043000240023004C000F00150006000A000900EC
:1004400038001600110017000B00070028001D00DF
:1004500019001A00100005004F0052005100500012
:1004600024522C0035021E021F0220022102220209
:1004700035021E021F022002210222024C003A0015
:100480003B003C003D003E0005784000410042003A
:1004900043004400010001000100010001000100CF
:1004A0002A00270226022502240223024C002702EA
:1004B0002602250224022302310230022F022E02DC
:1004C0002D023F0001004D004A0064023202450047
:1004D000AE00A900AA00AB000100010035001E001B
:1004E0001F0020002100220035001E001F002000F8
:1004F000210022004C003A003B003C003D003E0041
:10050000010040004100420043004400010001009E
:1005100001000100010001002A002700260025003B
:10052000240023004C00270026002500240023007F
:10053000310030002F002E002D003F0001004E0042
:100540004B00640032004500AE00A900AA00AB00D9
:10055000010001003A003B003C003D003E003F002E
:100560000100007C4278437846784578010001001C
:100570000100807481741570010001000100010008
:100580000100010001000100010001000100010063
:100590004500440043004200410040004C0001007F
:1005A00049784A7847784878010001004252415220
:1005B000405214700100010001000100010001001F
:1005C000010001000100010001000100FD377A581F
:1005D0005A000004E6D6B4460200210116000000CD
:1005E000742FE5A3E003B201085D003D888986D33E
:1005F000DC0AE842C3249258425AFA4B42162C5F56
:10060000542BA3199BCDF09E3ED52B7388208A27AF
:1006100002C28C6C91863337C68276CB812B45B073
:100620004557660343EA9B6B19E8B1AAA5E31F2C63
:1006300065784B4034F572DD554C0E88976FFB9210
:100640000FB4A5F05BB19A2B1D54928E8272F648BE
:10065000E7B4799F489284ADB1C6FC79939A8D1C1A
:1006600035FF1B43F6C6C36EBA331667230739003E
:1006700080DCF0C90C81E00A7D63DD01534C5B95A1
:10068000B69BDD20F18041788D582E31A49DE6E4A3
:1006900022C3AEFD3C42DB72E04C0613E4B985296F
:1006A000FF5AE82552FB2F1DAE76F50CE6A9333E26
:1006B000C260D50808F250A7490CB73F7F5CCCBB9D
:1006C0008B1564DEBF6F0059C9DDAAEC69D00951F2
:1006D000F1D362269E135492CC3819E51A9CEAD3C2
:1006E00022865F6703DF3AED5FB76A10E5AD968D4E
:1006F0004D7F0000B6C38E336581AEE60001A402D3
:10070000B3070000B4239031B1C467FB02000000BE
:100710000004595A11241FBECFEFDAE0DEBFCDBF6F
:1007200011E0A0E0B1E0EAEEF2E602C005900D9221
:10073000A23CB107D9F723E0A2ECB1E001C01D92C1
:10074000AE3EB207E1F70E942D260C94DA3058CC69
:100750009C019A9581159F4118F5F32FF270EE27B1
:10076000832F8170732F74706627532F587044271E
:1007700034FF0CC08295807FEF2B09F08062672BDD
:1007800009F08064452B69F080680895EF2B09F02B
:100790008260672B09F08460452B19F0886008950A
:1007A00080E00895CF93DF93EB01D2DFFE0109953E
:1007B000DF91CF910895982F92959F7024E0911129
:1007C00002C020E0982F892F86958695811511F01B
:1007D0002E5F982F892F8695820F08958093A3030B
:1007E00008958093A403089521E030E001C0220F12
:1007F0008A95EAF78091A403822BF3CF21E030E0C1
:10080000A90102C0440F551F8A95E2F7CA018095DD
:100810009091A4038923E5CF292F9A3090F5863053
:1008200080F590E036E0239F800D911D1124282F44
:10083000277041E001C0440F2A95EAF723E096951E
:1008400087952A95E1F7FC01EE0FFF1FE80FF91FCE
:10085000EF59FD4F20E030E070E05191DF01CB0116
:10086000022E02C0969587950A94E2F781708195D1
:100870008527842385278E932F5F3F4F23303105B3
:1008800061F70895292F9A3078F5863068F590E061
:1008900036E0239F800D911D1124682F677023E09F
:1008A000969587952A95E1F7FC01EE0FFF1FE80F5B
:1008B000F91FEF59FD4F40E050E080E0219130E01A
:1008C000062E02C0369527950A94E2F72170332749
:1008D000042E01C0220F0A94EAF7822B4F5F5F4F6C
:1008E0004330510559F7089580E008959091A4038D
:1008F00021E030E0F90101C0EE0F8A95EAF7D90155
:1009000002C0AA0FBB1F6A95E2F7EA2B01C0220FB3
:100910004A95EAF7892F8E23E81303C0892F822B8B
:1009200060CF2095822F8923FBCF8091AC039091DB
:10093000AB03981301C008958F5F8770FACF909131
:10094000A603809589238093A603282F2770211161
:1009500010C0891771F09091ED0392FF0AC086953F
:10096000869586954BDF1092A6031092A8031092ED
:10097000A70308959091A103982B9093A103089544
:10098000982F90958091A10389238093A1030895C6
:100990008091A003811531F01092A0031092AA0358
:1009A0001092A9030895803E9105D9F1C8F48133CE
:1009B000910509F482C048F48932910509F472C0A6
:1009C0008A32910509F480C0089589339105E9F0D0
:1009D00082389105D1F08533910509F45EC0089500
:1009E000843E9105D9F148F4823E910539F1833E68
:1009F000910549F181EE90E00895863E9105C9F197
:100A0000873E910509F43EC008952091EC032370C0
:100A1000211164C02091ED0323FF14C089E290E00E
:100A200008952091EC0320FD45C03091ED0330FF87
:100A300009C024FD24C083EE90E008952091EC03CA
:100A400022FDF7CF08952091EC0322FD44C03091A0
:100A5000ED0330FD43C024FFF5CF11C02091ED031D
:100A600021FFF0CF8091EC0384FD09C087EE90E078
:100A700008952091EC0323FFE5CF24FFF7CF80E01A
:100A800090E008952091EC0323FD2BC03091ED03FD
:100A900031FFE1CF84EE90E008952091EC0325FF33
:100AA000D1CFBCCF2091EC0325FD1EC02091ED03DA
:100AB00023FFC8CF89E390E008952091EC0326FF3F
:100AC000C1CF8AE290E008952091EC0326FFBACFCF
:100AD00081E390E0089582EE90E0089580EE90E04A
:100AE000089586EE90E0089585E390E00895909152
:100AF000EC0392FF10C041E0282F2471243009F04C
:100B000040E031E0282F2871283009F030E0431709
:100B100011F02CE0822793FF10C041E0282F2471B0
:100B2000243109F040E031E0282F2871283109F004
:100B300030E0431711F02CE082273091ED0330FFB5
:100B400010C051E0282F2171213009F050E041E020
:100B5000282F2871283009F040E0541711F029E0BF
:100B6000822731FF10C041E0282F2171213109F087
:100B700040E031E0282F2871283109F030E0431798
:100B800011F029E0822794FD877E08951F93CF936B
:100B9000DF9309DFEC01811522E5920708F052C0CE
:100BA000811540E5940708F0CDC0803E910520F501
:100BB0008D3C910508F0A1C0883A910570F4853A02
:100BC000910508F097C081309105B9F10497813AF9
:100BD000910598F1C0E0D0E030C0885A91094B9758
:100BE000C8F7C85AD0E0CC0FDD1FCB5ADE4F0990B2
:100BF000D881C02DD46421C0811550E49507B0F48C
:100C0000C11580E2D80708F0B3C0C83ED105A8F0EE
:100C1000CE019A9581159F41E8F68D2F68DF182F38
:100C2000CE019927C0DEEC01D12B07C09927BBDE8E
:100C3000CC27DF70C82BD92BD06ACE01DF91CF91A2
:100C40001F910895803842E59407C8F5803652E533
:100C5000950708F05BC0C03482E5D807D0F4C032F5
:100C600092E5D90708F04BC08C2F8695869520E237
:100C7000829FC0011124C37021E030E0A90102C0AD
:100C8000440F551FCA95E2F7EA01C82BD92BDD683E
:100C9000D4CF8C2F86958695877050E2859FC001B2
:100CA0001124C37021E030E0A90102C0440F551F98
:100CB000CA95E2F7EA01C82BD92BDC68BECF803C8D
:100CC00052E5950758F48F71C03AD245A0F590E0EF
:100CD000982F8827EC01C46FD06AAFCF805C924513
:100CE000809708F077CFDC2FCC27CC27DF71C06F3F
:100CF000D06AA3CFA497D064A0CFD0659ECFCF7188
:100D0000D0E0DC2FCC27C16FD06A97CF869586952F
:100D1000877020E2829FC0011124C37021E030E07F
:100D2000A90102C0440F551FCA95E2F7EA01C82B7A
:100D3000D92BDA6882CFDBDEC82FD0E0DC2FCC27BE
:100D4000D0627BCF8F71D3DE93E0CC0FDD1F9A95FD
:100D5000E1F7CC27DF70282F30E084FF05C050E199
:100D6000859F900111243327C22BD32BD06965CFE7
:100D70008D2F8F71BCDE182FCE01992714DEEC0168
:100D8000D12BDECF80E00895F894E82FE295EF7044
:100D9000F0E041A18F7021E030E0B90102C0660FA0
:100DA000771F8A95E2F7CB01962F9095942391A314
:100DB00092A1892B82A37894089581152CE792073C
:100DC00041F42091310230913202232B11F480E062
:100DD00090E00895E9E1F3E080E090E06BE475E2F3
:100DE0004EE655E220EE35E27783668351874087F1
:100DF000338722879787868701967096883091057A
:100E000099F70895FC018481862381110AC08281AB
:100E10008115B9F06823908593FF05C081E06111C9
:100E20000FC080E00895282F22952F708F70282BF7
:100E3000962F92959F706F70962B81E02913F1CFBA
:100E4000089581E008950F931F93CF9301E010E080
:100E5000082E01C0000F0A94EAF7C0919F039C2F4F
:100E60009023911115C09091A6039695969596950D
:100E7000891306C01092A6031092A8031092A7032C
:100E8000B3DCC027C0939F03CF911F910F910895AA
:100E9000B5DCF7CF282F35EB2303C001112497FFD2
:100EA00004C080589109892F089580589F4FFBCF27
:100EB00080917F0280FF0DC060912C0170E0660F71
:100EC000771F60387105B0F561157105A9F1862F9E
:100ED000089581FF07C060912C0184E0689FB001F4
:100EE0001124EFCF82FF04C060912C0188E0F6CF7F
:100EF00090917E029115D9F020912B0180912C01C7
:100F0000682F70E0921730F043E0660F771F4A9524
:100F1000E1F7D7CF899FC001112433E0880F991FD3
:100F20003A95E1F7622F70E00E941F30CACF68E067
:100F300070E0CDCF8FE7089581E0089580917F0222
:100F400080FF0CC060912A0170E0759567957595DA
:100F500067956115710549F1862F089581FF06C0D7
:100F600060912A0170E075956795F3CF60912A0131
:100F700082FD0BC090917D029115A1F06091290135
:100F800080912A01961738F0682F70E0603871055B
:100F900000F38FE70895899FC001112470E00E943B
:100FA0001F30F4CF61E070E0D7CF81E00895FA01FF
:100FB000309709F00995089580914B02811569F0E9
:100FC000E0915702F0915802309739F00190F0818A
:100FD000E02D309711F00995089580E00895A3E081
:100FE000B0E0E5EFF7E00C94F82F9C018091F2015E
:100FF0009091F30182179307B1F03093F30120939E
:10100000F201E0915702F0915802309761F00084AC
:10101000F185E02D309739F083E089833B832A8383
:10102000CE01019609952396E2E00C941430A3E0DA
:10103000B0E0EDE1F8E00C94F82F9C018091F00114
:101040009091F10182179307B1F03093F101209351
:10105000F001E0915702F0915802309761F000845E
:10106000F185E02D309739F084E089833B832A8332
:10107000CE01019609952396E2E00C941430A6EC7B
:10108000B1E0EFEF90E02D91821751F0EF3F19F4AE
:10109000211101C0E92F9F5F9630A9F7EF3F09F4B6
:1010A00008950E2E000CFF0BEC53FE4F8283089523
:1010B000E6ECF1E09191891302C0DF011E9291E00C
:1010C000EC3CF907B9F708958091010108952FB715
:1010D000F8948091EC019091ED01A091EE01B09116
:1010E000EF012FBF0895962F2091ED0322FF0EC030
:1010F000682F660F660F660F692B6093A60374DB7B
:10110000E6DF9093A8038093A70308956DCB909199
:10111000A003292F2823211559F080958923809336
:10112000A003811531F0D3DF8093A9039093AA0324
:10113000089580E090E0F8CFCADF209182023091DC
:101140008302232B211521F080932002909321020A
:101150002091840230918502232B211521F0809368
:101160001E0290931F02E0915702F09158023097AF
:1011700059F00680F781E02D309731F082E08093BE
:10118000800280E892E009950895611509F441C054
:10119000E3E3E80FE33148F4F0E0E452FF4C0C9451
:1011A000323086DE819580938302C6CF81DEFBCF0D
:1011B0007FDE819580938202F8CF7ADEFBCFBEDEA0
:1011C00080938402F2CFBADE8195FACFB7DE8195A3
:1011D00080938502EACFB2DEFBCF815D990B21E0DF
:1011E00030E001C0220F8A95EAF780918102822BBC
:1011F00080938102DACF80917F02816080937F02A9
:10120000D4CF80917F028260F9CF80917F02846089
:10121000F5CF409182028D3C59F48091830287FF83
:101220000DC010928302411559F410927E0208C03D
:101230008E3C81F48091830218169CF3411581F055
:101240008091840290918502892B8111AECF1092FA
:101250007D02ABCF8F3C41F447FFF0CF109282026A
:10126000809183028115E0CF803D19F41416B4F308
:10127000E5CF90918402893D29F41916FCF610926D
:101280008402DCCF8A3D19F497FFD8CFF8CF909134
:1012900085028B3D29F497FFD1CF10928502CECFE6
:1012A0008C3D19F41916CCF3C9CF9FE2980F9830F2
:1012B00090F4815D990B21E030E0B90102C0660F26
:1012C000771F8A95E2F7CB0180959091810289235F
:1012D00080938102B3CF8D3D31F480917F028E7F68
:1012E00080937F02ABCF8E3D21F480917F028D7F72
:1012F000F7CF8F3D09F0A2CF80917F028B7FF0CF97
:101300002FB7F8946091EC017091ED018091EE019E
:101310009091EF012FBF08950F931F9380914B027F
:10132000811521F0EDDF1F910F910895E9DF009104
:101330004D0210914E0220914F0230915002600FE9
:10134000711F821F931FEFCFCF92DF92EF92FF9218
:10135000CF93DF93D82FC92FC0901303D0901403DD
:10136000E0901503F0901603CBDF6C197D098E0910
:101370009F09643F71408105910510F1C1DF6B0148
:101380007C0182E390E0A0E0B0E0C0921A02D0922B
:101390001B02E0921C02F0921D02809316029093B1
:1013A0001702A0931802B0931902D0931103C093AF
:1013B0001203DF91CF91FF90EF90DF90CF900895CF
:1013C00084EF91E0A0E0B0E0E0CF87E797E790936B
:1013D00001088093000888E19AE00FB6F894A89578
:1013E000809360000FBE90936000FFCF0895FC01D2
:1013F0009B018091E2019091E3018617970740F0ED
:10140000672B29F48091E8008E778093E800C9016A
:1014100040E0009741F4411106C08091E80082FF4E
:101420002FC080E00895209133022115A9F12530C5
:10143000A9F12091E80023FD2DC02091E80022FDB4
:10144000ECCF2091E80020FFE4CF3091F300209111
:10145000F200009719F02830310558F041E02830AB
:10146000310509F040E02091E8002E772093E80054
:10147000D0CF41914093F10001972F5F3F4FE9CFCB
:1014800080913302811541F0853041F08091E80070
:1014900083FFC3CF81E0089582E0089583E008953B
:1014A0008091DC0187FF13C08091E80082FF06C0B5
:1014B0008091E8008B778093E80008958091330253
:1014C0008111F2CF0895809133028115D9F3809173
:1014D000E80080FFF8CF8091E8008E77ECCF209174
:1014E000E4003091E50095E6A9012091EC00822FFF
:1014F000817020FF06C08091E80080FF06C080E078
:1015000008952091E80022FD1AC0809133028115D0
:1015100089F0853089F08091EB0085FD0FC0209126
:10152000E4003091E50042175307F9F29A95E1F68D
:1015300084E0089582E0089583E0089581E00895AD
:10154000E8EDF0E080818E7F80831092E2001092BF
:10155000DA001092E100A0EEB0E08C9181608C93F3
:1015600080818F77808319BCA7EDB0E08C918E7F4E
:101570008C9380818F7E80831092DB010895E091AF
:101580005702F0915802309739F00284F385E02D2C
:10159000309711F060E209950895FC01AC014B5FB2
:1015A0005F4F8FEF61E39191892728E030E0982F1A
:1015B000990F87FF09C0892F862721503040B9F73E
:1015C000E417F50781F70895892FF7CF982F9093A7
:1015D000E900891771F07091EC002091ED005091B5
:1015E000F00021FD09C09F5F973089F78093E900E3
:1015F0000895762F242F50E03091EB003E7F3093FA
:10160000EB003091ED003D7F3093ED003091EB0029
:1016100031603093EB007093EC002093ED00509319
:10162000F0002091EE0027FDDECF0895A0E0B0E0AD
:10163000ECE1FBE00C94F22FC8EDD0E088818F7EC6
:101640008883E7EDF0E080818160808384E082BF61
:1016500081E08093DB0188818E7F888302EE10E039
:10166000F80110821092DA0081EEC82ED12CF6011A
:10167000108288818F7788838881806888838881B9
:101680008F7D888319BC109233021092DA01109278
:101690000A021092D90190EEE92EF12CF701808117
:1016A0008B7F808388818160888342E060E080E076
:1016B0008DDFF60180818E7F8083F80180818160DB
:1016C0008083808188608083F70180818E7F808322
:1016D000888180618883CDB7DEB7E8E00C940E3056
:1016E000E091AC039091AB0327E0E91302C080E0E6
:1016F0000895AE2FB0E02E9FF0011124E355FC4F6A
:101700003181361306C03081381303C0358134135C
:1017100004C0FD013196E770E8CF81E008950F9392
:101720001F93CF93DF938B01EA01909133029430A2
:1017300051F58093E9008FEF9091E80095FD06C088
:1017400095ED9A95F1F700008A95B1F78091E80040
:1017500085FF19C0C4DE811111C08091E80085FDAC
:1017600006C08091E8008E778093E800F3CFF801FF
:1017700081918F018093F100219779F78091E800A2
:101780008E778093E800DF91CF911F910F9108959C
:10179000792F603229F440E250E0682F82E0BFCF19
:1017A0000895CF93DF93D82FC92F48E050E0682FDA
:1017B000792F81E0B4DF88E0ED2FFC2FA4EEB1E0BB
:1017C00001900D928A95E1F7DF91CF910895BC01C8
:1017D00046E050E084E0A3CFBC0143E050E084E069
:1017E0009ECFA0E0B0E0E7EFFBE00C94F02FF82EE6
:1017F000E92EB62EA72E8A018091D6019AE0C92E35
:10180000D12C8A3018F0CC24C394D12CC1E0D0E084
:101810006B2D7A2D8F2D9E2DF8010995811116C003
:101820002196CC16DD0694F0CC9FC001CD9F900D83
:10183000900D112420E030E045E34A95F1F70000D7
:101840002F5F3F4F28173907B9F7E2CFCDB7DEB783
:10185000EAE00C940C30CF93DF93C1E0D0E001C0FC
:10186000CC0F8A95EAF76C2F83E090E00E94A530B8
:101870008C2F0E94EE03DF91CF9108951F93CF9399
:10188000DF93962F122F632F8630D8F49A30C8F446
:101890004630B8F4C42FD0E0CC0FDD1F2CE0929F6F
:1018A000C00DD11D112498E7899FC00DD11D1124B1
:1018B000CE0189960E94A530612FCE018A960E94A2
:1018C000A530DF91CF911F9108959091ED0392FB88
:1018D000222720F9281771F080FB92F99093ED03ED
:1018E0006091EC037091ED0384E090E00E94BF30C2
:1018F00082E025C80895CF93DF93C091A103809122
:10190000A503C82B8091A0038115E1F0E0DB2091B5
:10191000A9033091AA03821B930B8838934108F0E6
:1019200037D8D091A00320E086EC91E0FC01308113
:10193000019631112F5F31E08C3C9307B9F72111EB
:1019400027D8CD2B8091950280958C23909194027D
:10195000892B8093C40148E050E069E572E084EC93
:1019600091E00E945C30892BB9F088E0E4ECF1E072
:10197000A9E5B2E001900D928A95E1F7E091570256
:10198000F0915802309741F00280F381E02D3097BA
:1019900019F084EC91E00995DF91CF910895CF93F0
:1019A0001092A103C6E0E6ECF1E0DF018C2F1D925E
:1019B0008A95E9F780E090E012DB80E090E037DB89
:1019C0001092A50398DFE0E8F2E0DF011D92CA95CE
:1019D000E9F710927E0210927D0210927F02ACDB3A
:1019E000CF910895DCDF2FEF84E39CE0215080400D
:1019F0009040E1F700C0000088E19AE00FB6F8944B
:101A0000A895809360000FBE90936000FFCFAAE27C
:101A1000B0E0EDE0FDE00C94F72F8CED91E0FC01DF
:101A200001962091F100208321E0843E9207B9F7CE
:101A30008091DD01893009F457C0C8F4823009F47F
:101A4000B2C0833009F482C0813081F18091E80016
:101A500083FFE6C08091DC019091DD019A3008F0AF
:101A6000DFC0E92FF0E0E151FF4C0C9432308A30B6
:101A700009F489C08B3051F78091DC01813231F754
:101A80008091E0019091E101892B01F78091E800BC
:101A9000877F8093E80004DD81E09091DE01911161
:101AA00001C080E0809302017ADFD0CF8091DC0119
:101AB000813A61F68091E800877F8093E800809109
:101AC000E0019091E101892B59F060E080E090E025
:101AD00070E08DDC8091E8008B778093E800B6CFD2
:101AE00068E084EE91E0F4CF8091DC01813209F06E
:101AF000ADCF8091E0019091E1018D7F892B09F0BC
:101B0000A5CF8091E800877F8093E8008091E8006E
:101B100082FF17C09091F3008091F200029731F498
:101B20008091F100813011F0863021F48091F10034
:101B3000809301018091E8008B778093E800B0DC0E
:101B400085CF809133028111E1CF80CF8091DC017C
:101B5000813A09F07BCF8091E0019091E101892BDE
:101B600009F074CF8091E800877F8093E80080912E
:101B7000E80080FFFCCF809102018093F10080910A
:101B8000E8008E77DACF8091DC01813209F05ECFF8
:101B90008091E800877F8093E80082DC8091DF01FC
:101BA0008093000153CF8091DC01813A09F04ECF40
:101BB0008091E800877F8093E8008091E80080FFB3
:101BC000FCCF80910001D9CF803889F0823841F56F
:101BD0008091E0018F70873018F58093E900809143
:101BE000EB0085FB882780F91092E90006C0809100
:101BF0000A02880F9091D901892B9091E800977F74
:101C00009093E8008093F1001092F1008091E80039
:101C10008E7723C0811116C08091DE01813009F1D9
:101C20008091E80083FF0AC08091E800877F80935D
:101C3000E8008091EB0080628093EB00AA96E3E0DD
:101C40000C941330823061F78091DE01811581F0B0
:101C50001092E9008091E800877F8093E80020DC03
:101C6000DFCF81E0933009F080E080930A02F0CF6B
:101C70008091E0018F702FEF280F263088F6809337
:101C8000E9002091EB0020FFE3CF933031F4809105
:101C9000EB0080628093EB00DBCF9091EB009061D2
:101CA0009093EB0021E030E0A90102C0440F551FE2
:101CB0008A95E2F74093EA001092EA008091EB00E7
:101CC0008860E8CF8111ACCF1091DE011F77809141
:101CD000E3008078812B8093E3008091E800877F88
:101CE0008093E800DDDB8091E80080FFFCCF8091ED
:101CF000E30080688093E30083E0111101C082E07B
:101D0000809333028DCF8058823008F089CF809144
:101D1000DE019091DF018C3D53E0950791F583E062
:101D20008A838AE289834FB7F894DE01139620E014
:101D30003EE051E2E32FF0E050935700849120FF02
:101D400003C082958F703F5F8F708A30C0F0895CCE
:101D500090E08D939D932F5F243161F74FBF809169
:101D6000E800877F8093E8006AE270E0CE01019688
:101D70003EDB8091E8008B778093E80051CF805D57
:101D8000E7CF292F33272330310509F44EC078F5EA
:101D90002130310509F488C08BE590E0EDE3F2E0F5
:101DA0002230310509F03CCF2091E800277F2093B5
:101DB000E8002091E2013091E3018217930708F4D3
:101DC0009C0140E02115310509F073C0411171C03B
:101DD0008091E80082FDCDCF80913302811549F2D8
:101DE000853039F28091E80083FFF2CFC2CF809135
:101DF000E0019091E1012132310509F446C022321F
:101E0000310509F00DCF8330910508F009CFFC01B1
:101E1000EE0FFF1FE45CFE4F0190F081E02D875C28
:101E20009E4FDC018C9190E010C09C0133278230E2
:101E300021F12330310568F4232BB9F4E8EFF2E007
:101E4000E4918E2F90E0E8EFF2E0009709F4E8CEFD
:101E5000ABCF2330310509F0E3CEEAEAF2E0E491BA
:101E60008E2F90E0EAEAF2E0F0CFE8EEF2E0E491C3
:101E70008E2F90E0E8EEF2E0E8CFE8ECF2E0E491BB
:101E80008E2F90E0E8ECF2E0E0CF8330910508F08F
:101E9000C7CEFC01EE0FFF1FEE5BFE4F0190F081FD
:101EA000E02D89E090E080CF82E190E0E8E9F2E087
:101EB0007BCF80913302811509F45BCF853009F423
:101EC00058CF8091E80083FD54CF8091E80082FDD7
:101ED0007FCF8091E80080FF75CF9091F3008091D3
:101EE000F2002115310519F08830910550F041E0DC
:101EF000089709F040E08091E8008E778093E80031
:101F000061CF44914093F1003196215031090196FF
:101F1000E8CF803809F084CE8091E800877F8093F5
:101F2000E8008091DA018093F10070CE811178CEC3
:101F30001091DE01123008F073CE8091E800877FA7
:101F40008093E8001093DA01ABDA1115D9F084E040
:101F50008093330242E061EC81E038DB42E261ECE5
:101F600084E034DB42E261EC82E030DB42E260ECB0
:101F700083E02CDB80913302843051F482E0809343
:101F800003014ECE8091E30087FDE1CF81E0E0CFF9
:101F900081E0F5CF811509F447C0823849F40CD8A7
:101FA00081FF42C089E36BD8A6DC89E381D8A3CC4A
:101FB000833841F401D880FF37C083E560D89BDCCB
:101FC00083E5F4CF843849F40E94DC0782FF2CC0FB
:101FD00087E455D890DC87E4E9CF9CEF980F913ADD
:101FE00028F390E2980F983050F4877091E001C088
:101FF000990F8A95EAF7892F0E94C004D8CF9BE5F4
:10200000980F933020F480E090E00C94EF0798E56F
:10201000980F9B3118F480E090E009C893E3980F83
:10202000933110F460E0B1C80895811519F00E9451
:10203000BA0461CC0895811519F00E94C0045BCCEC
:102040000895811531F09091A503892B8093A50304
:1020500052CC0895811539F080959091A50389237C
:102060008093A50348CC089580919002811521F0BA
:1020700082E2F0DF109290020895CF93DF93EC019B
:102080004A855B856E857F850E94D7079B819095E9
:102090008091A50389238093A5038C810E94C004AD
:1020A0002ADC86E0FE0111928A95E9F7DF91CF9153
:1020B0000895CF93DF93EC018D8181FD13C0826081
:1020C0008D838091A5039B81892B8093A5038C81AF
:1020D0000E94BA0410DC488559856E857F85CE0143
:1020E0000E94D70710929A03109299038D8180FD68
:1020F00002C0CE01C2DFDF91CF9108951F93CF932D
:10210000DF93182FA0910F03B0911003109709F4DB
:1021100048C010921203109211031092950210926F
:1021200094021696CD91DC911797CE019A95811560
:102130009F4108F4D07ED1E0C11101C0D0E01996D2
:10214000ED91FC911A97309731F01B966D917C912F
:1021500080E00995D823D11539F08CEF8C0F813AA6
:1021600020F58C2F0E9458081115A1F0E0910F0363
:10217000F0911003808584FD0DC080910E038115C0
:1021800049F0808191819C01215031092F333E47D4
:1021900008F4DAD8B0DB1092100310920F031092FB
:1021A0000E03DF91CF911F910895A5DB8C2FF2DEF6
:1021B000DBCFAFE0B0E0EFEDF0E10C94EB2FFE01F0
:1021C00031968AE0DF011D928A95E9F788E4E82ECE
:1021D00081E0F82E8F019DE4C92E91E0D92E3F01B8
:1021E000AA24A394B12C33E5832E31E0932EF7017A
:1021F00081917F018F3F09F43EC0F894E82FE2956A
:10220000EF70F0E021A18F70A50102C0440F551FAF
:102210008A95E2F7CA01922F982B91A392A18095FB
:10222000892382A3789400C0EDE4F1E031E0512CE1
:1022300021912F3F79F0A22FA295AF70A05EB0E060
:102240008C9190E02F7002C0959587952A95E2F7C2
:1022500080FF73C080E0582A330F8E169F0641F727
:10226000F70182918F3F11F00E94C40650EA5A95FF
:10227000F1F7D8015C920F5F1F4FCE14DF0409F015
:10228000B6CF4AE050E0B3018DEF91E00E945C30A0
:102290009C01892B41F08AE0F301ADEFB1E00190A0
:1022A0000D928A95E1F70091080210E0095D1D4F3B
:1022B000232B09F444C081E08093D5010E94670874
:1022C0009093D4018093D30180914B02811509F43E
:1022D00090C07E01BBE0EB0EF11C85E0F70111928E
:1022E0008A95E9F78091D6018A3008F04CC04EE813
:1022F00052E1B701C80175DA811509F468C043E3FA
:1023000052E1B701C8016DDA811509F460C010927D
:10231000D6018091070290E045E050E0B701895D69
:102320009D4F0E945C3021E02093D201892B09F05F
:1023300041C02F96EFE00C940730832F8CCF809113
:10234000D501811509F4C0CFE090D301F090D401FC
:102350000E9467088E199F09059708F4B5CF45E0DC
:1023600050E06DEF71E0C8010E945C30892B41F0B4
:1023700085E0EDEFF1E0D80101900D928A95E1F74B
:102380001092D501A1CFC090D001D090D1010E9470
:1023900067088C199D09843F914008F0A8CF80916F
:1023A000D201811531F285E0D7011D928A95E9F7B6
:1023B0001092D201A0910702B0E0A95DBD4F85E067
:1023C000FE013B9601900D928A95E1F7B2CF809184
:1023D000D6018F3F39F40E9467089093D101809312
:1023E000D001DDCF8F5F8093D6018A3008F491CF82
:1023F000F2CF85E0F801A9E3B2E001900D928A9551
:10240000E1F789E392E0C9D880933802C0903E0298
:10241000D0903F02E0904002F09041028091CC01C8
:102420009091CD01A091CE01B091CF01C816D906EF
:10243000EA06FB0609F47DCFC092CC01D092CD0113
:10244000E092CE01F092CF010E948009C61AD70A0D
:10245000E80AF90AC0924D02D0924E02E0924F0271
:10246000F092500266CFCF92DF92EF92FF921F93CD
:10247000CF93DF9300D000D0CDB7DEB7C090340249
:10248000D0903502E0903602F09037020E94800929
:102490006C197D098E099F0911E06436710581056B
:1024A000910578F10E948C09DC01CB010296A11DF7
:1024B000B11D89839A83AB83BC8380912201909163
:1024C0002301885C9D4F20912101422F50E025304F
:1024D00010F044E050E0BE016F5F7F4F0E94693012
:1024E00082E090E00E947A2F182F811551F00E940F
:1024F0008009609334027093350280933602909382
:102500003702812F0F900F900F900F90DF91CF9196
:102510001F91FF90EF90DF90CF9008958F929F9240
:10252000AF92BF92FF920F931F93CF93DF9300D090
:1025300000D000D0CDB7DEB7F62E072F80E090E0B8
:102540000E947A2F182F811509F460C08091140120
:10255000482F50E0811511F041E050E060911501E5
:1025600070911601685C7D4FCE0106960E9469301D
:102570008090470290904802A0904902B0904A0291
:102580000E948009681979098A099B0964367105D6
:102590008105910538F489E392E00E94CD0A9E817D
:1025A0008917A1F181E090E00E947A2F8115C9F18D
:1025B00080911C01482F50E0863010F045E050E03B
:1025C00060911D0170911E01685C7D4FCE010196E6
:1025D0000E94693089E392E00E94CD0A9E818913AE
:1025E00020C00E9480096093470270934802809344
:1025F000490290934A0285E0FE013196A2E4B2E0DE
:1026000001900D928A95E1F781E00CC085E0E9E345
:10261000F2E0DE01119601900D928A95E1F7111119
:10262000EACF80E095E0E2E4F2E0AF2DB02F019038
:102630000D929A95E1F70F900F900F900F900F90D9
:102640000F90DF91CF911F910F91FF90BF90AF90AE
:102650009F908F9008950F931F93CF93DF938630B1
:1026600030F56A3020F5463010F5C42FD0E0CC0F9D
:10267000DD1F2CE0629FC00DD11D112438E7839F20
:10268000C00DD11D1124CE0189960E948930082FDA
:1026900010E0102F0027CE018A960E948930980101
:1026A000282BC901DF91CF911F910F91089580E0F0
:1026B00090E0F8CF462F672F2091530230915402BB
:1026C000232B81F4703F39F4403F61F48091510233
:1026D0009091520208957A3028F4463018F48630EA
:1026E00008F4B9CF80E090E00895A0E0B0E0EBE717
:1026F000F3E10C94F32F7C010091A4038091A303D8
:10270000082BC5E0D0E010E0C8010C2E02C0959562
:1027100087950A94E2F780FD09C02197A8F7D12C8C
:102720008D2DCDB7DEB7E7E00C940F30DC2EB7016E
:102730008C2FC0DF0E94C605019779F3F1CF0F936C
:102740001F93CF93FC01858100811181811581F058
:10275000611571F0C801C9DFC82F682FC8010E9438
:102760000C04B8018C2FA6DFCF911F910F91089513
:10277000C8010E944204C82FF4CFCF93DF93D82F13
:10278000C92FB3DF6D2F7C2F95DF0E94C605DF9127
:10279000CF910895FC018481811599F08081918108
:1027A000ECDF282F92959F70963099F060F4925F3D
:1027B0009F70923030F4203FB1F038F481E0283E31
:1027C00038F080E008959A5FF3CF81E0243FC9F7A5
:1027D000089591E0213F09F090E081E0283E08F063
:1027E00080E0892B089581E00895382F292FCB01AF
:1027F000A32FB22F87369105A105B10520F4875686
:102800009C4F0C94893080E0089585E290E00E940E
:1028100089308F3F89F486E290E00E948930823EC1
:1028200059F487E290E00E94893091E08E3D09F0F2
:1028300090E0892F8170089580E0FCCFAAE0B0E09D
:10284000E4E2F4E10C94ED2FC0903102D09032021A
:1028500081E090E09093320280933102812C912CA0
:10286000E12C5401F12C14C0F80125913591472D2C
:102870006F2D8E2D03D80E5F1F4F739486E0781254
:10288000F3CF96E0A90EB11CF394EAE0FE1639F0FE
:102890008501000F111F04501D4F712CE5CFE394EB
:1028A000FCE38F0E911C86E0E812DBCF1A821982BE
:1028B0001C821B821E821D8218861F8288EC90E07B
:1028C0009A87898709EF12E0FE0131967F014AE07D
:1028D00050E0B801C7010E94C330065F1F4F570187
:1028E0000934F3E01F0799F789E0F70111928A95FF
:1028F000E9F78FEF9FEF9E838D8387E08A874AE019
:1029000050E0B801C5010E94C330065F1F4F09396E
:10291000F3E01F07A1F7D0923202C09231022A964B
:10292000EDE00C940930AAE0B0E0E9E9F4E10C94A0
:10293000F02F06E912E089E4E82E83E0F82E97E014
:10294000B92E24EFC22E21E0D22EAA24A3944AE06D
:1029500050E0B701CE0101960E947930F801389617
:10296000DF018B2D1D928A95E9F789819A81D80123
:1029700011969C938E938F8112968C9312978D81D2
:1029800013968C931397888514968C931497898546
:1029900015968C9315978B819C8117969C938E939B
:1029A00016978A8587FD04C01E96DC92CE921D97ED
:1029B00080FF02C0F801A08681FF07C0D8011896E9
:1029C0009C911897926018969C9382FF04C0F8011E
:1029D00090859460908783FF07C0D80118969C91DA
:1029E0001897986018969C9384FF04C0F80190850E
:1029F0009061908785FF07C0D80118968C91189731
:102A0000806218968C93BAE0EB0EF11C015F1F4FA9
:102A1000E9E9EE16E3E0FE0609F099CF2A96EAE02E
:102A20000C940C30282FCB01283070F44AE0249FFE
:102A300090011124B90167507D4F4AE050E00E9497
:102A4000793080E090E008958FEF9FEF0895AAE03D
:102A5000B0E0EDE2F5E10C94F82F9C01975581155B
:102A6000914068F4BE016F5F7F4F822FDBDF892BBF
:102A700031F489859A852A96E2E00C94143088EC2A
:102A800090E0F9CFA0E1B0E0E8E4F5E10C94EA2FA2
:102A9000FE01319680E1DF011D928A95E9F707E09A
:102AA00010E099E9A92E93E0B92E27E6422E512C89
:102AB000612C712C4F0173016201B1E14B1651047D
:102AC000610471041CF080E1C82ED12CA601B5016F
:102AD000C4010E949630AC0CBD1C0D2C000CEE08FD
:102AE000FF084C185D086E087F080150104019F768
:102AF0006096E0E10C9406306FEF85E290E00E9472
:102B0000A5306FEF86E290E00E94A5306FEF87E27C
:102B100090E00E94A53060E088E290E00E94A5303D
:102B20008DDEB0DF6FEF85E290E00E94A53062EEAF
:102B300086E290E00E94A5306EED87E290E00C9472
:102B4000A53063EE7EEF80E090E00E94BF3060E051
:102B500082E090E00E94A53081E08093A30361E0D1
:102B600083E090E00E94A53060E074E184E090E0B2
:102B70000E94BF30C1DF40E050E0BA018FE090E03A
:102B80000E94B73040E050E0BA0183E190E00C943D
:102B9000B730982F8B3258F4853098F0EBEFE80F70
:102BA000E63278F4F0E0E750FF4C0C943230833496
:102BB00050F48A3308F060C0853339F081E09833EF
:102BC00009F080E008958334E1F781E00E94EE038C
:102BD0000E94CF0C01C0B5DF81E0089580910B0207
:102BE000807F80930B0281E080937C02F5CF8091FF
:102BF000310290913202892B79F30E94CF0C2FEF92
:102C000084E39CE0215080409040E1F700C0000048
:102C10000E94E50990910B02892F8E7F90FF8160C1
:102C200080930B0280FDD8CF817F80930B02D4CF9D
:102C300090910B02892F8D7F91FF826080930B0210
:102C400081FFCACF80910B028160EFCF90910B0280
:102C5000892F8B7F92FF846080930B0282FDF2CFDD
:102C6000BBCF90910B02892F877F93FF8860809361
:102C70000B0283FDE7CFB0CF995381E001C0880FED
:102C80009A95EAF7A3CF9D51F8CFCF93C82F81151E
:102C9000C9F08238C9F40E94DC0781FD13C089E3C2
:102CA0000E943F080E947B0C2FEF37EE83E02150FB
:102CB00030408040E1F700C0000089E30E945808DE
:102CC0000E947B0CCF9108958338A1F40E94DC0709
:102CD00080FDF8CF83E50E943F080E947B0C9FEFA8
:102CE00021EE34E0915020403040E1F700C0000078
:102CF00083E5E4CF8438A1F40E94DC0782FDE2CFB3
:102D000087E40E943F080E947B0C8FEF91EE24E045
:102D1000815090402040E1F700C0000087E4CECF12
:102D20008CEF8C0F813A08F0B3C080917C02813027
:102D3000D1F0823089F181112CC08091A1038232BF
:102D400021F48C2F26DF8111BDCFE6ECF1E08191DB
:102D5000C81709F4CDC081E0EC3CF807C1F78C2F0F
:102D60000E943F08ADCF8091A103823251F3C4315C
:102D700081F048F4CB3009F4A5CFC03131F782E0BF
:102D800080937C029FCFC93221F0C83309F49ACFD7
:102D9000DCCF10927C02D9CFCF3409F46FC0C0F4DD
:102DA000C832A0F4CE3198F5C73009F454C0C4310C
:102DB00009F088CF80917B02811509F483CF1092AE
:102DC0007B0210927A02109279027CCFC932F0CF46
:102DD000C13509F455C0C23509F454C086EFC03579
:102DE00009F070CFE0917902F0917A02309709F4FE
:102DF00069CF2081082E000C990B820F911D81153F
:102E000031E093070CF440C08FEF80835BCFCD514E
:102E1000C0937B02C430C9F078F48DE291E0C230F7
:102E200031F08EE291E0C33011F48CE291E09093A6
:102E30007A028093790246CFC53051F089E291E061
:102E4000C630A9F310927B023DCF8BE291E0EFCF29
:102E50008AE291E0ECCF81E080932E0184E18093BF
:102E60002D018AE080932C018EE180932B0188E074
:102E700080932A0188E28093290124CF8AE0B2CF8F
:102E80008FEFB0CF81E0AECF97FFBFCF10821ACFC8
:102E900080E28C0F883048F4C77081E001C0880F51
:102EA000CA95EAF70E94BA040BCF8BE58C0F8330EA
:102EB00038F42C2F2452330BC9010E94EF0702CFA4
:102EC000E8E5EC0FEB3150F4F0E0EE0FFF1FE557B3
:102ED000FE4F808191810E941708F4CE83E38C0F0E
:102EE000833108F0EFCE61E08C2F0E94C508EACE56
:102EF0008C2F0E9458080E947B0C31CFCF93DF9318
:102F0000EC01805E9109089720F061E270E1209762
:102F100011F465E170E1CE010E94D2038C2FB5DE81
:102F2000DF91CF9108951F93CF93DF93182FEB017B
:102F3000ACDE209731F4812F2DD8DF91CF911F91F6
:102F400008958FE99FE00197F1F700C000002197F5
:102F5000F0CFA0E0B0E0EFEAF7E10C94F32F162FEA
:102F6000D72FC42FD22E8115A1F040939D030E942C
:102F700067089093D8018093D701C77081E001C0A2
:102F8000880FCA95EAF751D8CDB7DEB7E7E00C94C1
:102F90000F3090919D03491335C0E090D701F09018
:102FA000D8010E9467089C012E193F097901812FE1
:102FB0009D2F4DDDE816F90628F5D0E2DD0DCD1583
:102FC00091F0C77011E0812F01C0880FCA95EAF710
:102FD00032D8D83040F48D2D877001C0110F8A95FA
:102FE000EAF7812F22D860E070E0802F9CDFD83094
:102FF00058F62D2D277081E001C0880F2A95EAF739
:103000001AD8C2CFC77081E001C0880FCA95EAF70D
:10301000F7CFA0E0B0E0EFE0F8E10C94F12FEC0185
:103020008881811511F1813009F046C08981813094
:1030300051F48A81239660E570E0893311F060E0F5
:1030400070E071DFEDCF823021F48A8123961DDE9E
:10305000E7CF833029F48A8123960E94CA0FE0CFFC
:10306000843041F022968111DBCFCDB7DEB7E9E0A5
:103070000C940D308A81239620E030E09AE0682F8E
:103080006053770BAB016A30710560F02115310593
:1030900051F3EFE9FFE03197F1F700C00000215054
:1030A0003109F4CF929FB001939F700D11249A01C2
:1030B000260F371F8991E3CFE82FF0E0E354FE4F4E
:1030C000B490282F26952695269530E0F901E355F2
:1030D000FE4FE4908770F12C082E02C0F594E7941F
:1030E0000A94E2F7E0FAEE24FF24E0F8F901E3564F
:1030F000FE4FC490D12C082E02C0D594C7940A94D8
:10310000E2F7C0FACC24DD24C0F8F901E357FE4F02
:10311000049110E002C0159507958A95E2F70170B9
:103120001127E114F10411F081EEAFDDC114D104D7
:1031300011F086EEAADD60E070E08B2DF4DEC114A4
:10314000D10419F086EE0E94CA0FE114F10419F0BF
:1031500081EE0E94CA0F0115110521F060E070E0B8
:103160008CE2E1DE21965CCFACE0B0E0EAEBF8E186
:103170000C94E92F7C01DC0114968C91811509F4E3
:10318000F5C061E0C701DBDA8C01F70185818115AB
:1031900029F18091990390919A030097F9F008170B
:1031A0001907E1F0FC01FF27887F9927892B09F097
:1031B0008AC0A4E0EE0FFF1FAA95E1F7E75EFC4F7F
:1031C00085818460858311830083CF010E9459101B
:1031D0001092A50361E0C701B2DA8C010034F2E578
:1031E0001F0709F483C008F071C0043232E51307E9
:1031F00009F49CC0053242E5140709F4A0C003326B
:1032000052E5150709F481C0D70115968C918115F7
:1032100009F43BC1C80197578038910508F0C4C133
:10322000003108F093C066E670E080E090E0DDDAFF
:1032300081118CC0812C912C540101119FC004E09C
:103240009E012F5F3F4F6901D601E02F1D92EA9545
:10325000E9F724013501FFEF4F1A5F0A6F0A7F0A71
:10326000C501B401C2DA8983811509F46FC08130C8
:1032700009F008C1A50194012E5F3F4F4F4F5F4FEA
:103280002D833E834F835887C301B201AEDA182FD6
:103290008A83811509F45AC08FEF810F833008F0BB
:1032A00086C06D817E818F8198859FDA8B838115A1
:1032B00011F0C601AEDE2401350133E0430E511C8E
:1032C000611C711C71C0E0E0F0E07ACF013482E54E
:1032D0001807A9F0023492E5190709F095CFD70134
:1032E00015968C91811591F182E006C0D701159653
:1032F0008C91811559F180E00E942B0C27C0F701B9
:103300008581811519F181E0F7CFF701858181155C
:1033100049F083E00E94F40345E064E083E00E940A
:10332000760414C083E00E94FE03F6CFD701159601
:103330008C91811511F084E0EDCF84E0F4CFF7019A
:1033400085818115B9F085E00E94F4038091A60380
:103350008770811559F0F7018581811539F08091C9
:10336000ED0382FF03C082E00E949F042C96E1E1FE
:103370000C94053085E00E94FE03E8CFB7E68B167B
:103380009104A104B10411F3C501B4012EDAEFEFE9
:103390008E1A9E0AAE0ABE0A8111F0CF01504DCF9F
:1033A0004D805E806F807884530142014DCF8BEF5A
:1033B000810F833090F52401350143E0440E511C08
:1033C000611C711C6D817E818F8198850EDA8B83E3
:1033D000811551F3C301B20108DA8C83811108C051
:1033E0002401350154E0450E511C611C711CDCCFD9
:1033F0008B819C818130AFEF9A0710F0982F88273E
:10340000163029F0173031F00E944025E9CF0E9494
:10341000ED24E6CF0E940E25E3CF143009F0C0CF93
:103420006D817E818F819885E0D9182F2401350127
:10343000B4E04B0E511C611C711CC501B4016D5FE1
:103440007F4F8F4F9F4FD1D9111509F47FCF811531
:1034500009F47CCF8150990B4FEF489F9001499F11
:10346000300D1124E12FE150FF0B2E0F3F1F215093
:10347000310908F499CF8FE99FE00197F1F700C077
:103480000000F5CFC601C5DD8FCF0115A7E51A07EE
:1034900008F4A5C00115B8E51B0708F0D1C76801FD
:1034A000E7E5DE1A66E872E08C2DBCDA892B31F58F
:1034B000C601E4E0880F991FEA95E1F7FC01E75E99
:1034C000FC4F2281213009F05AC0209186023091B0
:1034D0008702232B99F02091880230918902232BB7
:1034E00069F020918A0230918B0240918C025091B8
:1034F0008D02242B352B232B09F44BC08091900295
:10350000811509F4F1C0C090A103D090A0030E94DE
:10351000670888579C4E9093920280939102F7011E
:103520008581811509F4E0C08D2D8C298D7981115B
:103530000EC10115F0E51F0708F0A8C0011520E431
:10354000120708F00BC1063E110509F4CDC0C801F1
:1035500090528115904208F008C1D70116968C91BF
:10356000803108F4ECC0C80199271092A5038D3270
:10357000910509F0A4C082E08093A503FAC022302F
:1035800009F0BCCF20918A0230918B02232B09F4E1
:10359000B5CFFC01E25EFC4F20812E7F2083875E49
:1035A0009C4F0E945910AACF0337FCE71F07B9F4BC
:1035B00080919002811519F00E943410C7CE1092AC
:1035C000A1030E94C8040E94670888579C4E9093EC
:1035D00092028093910281E080939002B7CE023AEA
:1035E00022E51207C1F158F4C801905281159042AA
:1035F00018F1013E110579F1053E110503C0023BAA
:1036000052E5150709F07ACF25EE30E02770332711
:1036100081E090E001C0880F2A95EAF7209193029B
:10362000309190023115F9F0F70135813115B1F083
:10363000282B209393028ACED70116968C91803145
:1036400008F05CCF812F99278F71992782309105DF
:1036500011F04297D7CF21EE30E0D8CF809582236A
:103660008093930273CE322F3823311509F446CF5D
:10367000982F90959223909393020E94C004D701B3
:1036800015968C91811509F461CE38CF003EB2E5D4
:103690001B0708F047C0003CE2E51E0728F5003A8A
:1036A000F2E51F07E8F4003622E51207E8F4C80146
:1036B000925580349105C0F01092A503C8018E3256
:1036C000910508F063C08832910508F050C08E3132
:1036D000910508F04EC004974A9708F44CCF37C0C4
:1036E000043B32E5130741F7F7013580311409F443
:1036F00057C00E35FCE71F0709F44EC00F352CE705
:10370000120751F00D353CE7130709F049C08091CD
:103710002F01811509F440C010922F0180E00E9412
:103720007E1014CE09374CE7140728F407375CE7FE
:103730001507D0F6C1CF0B378CE71807D4CF812FF0
:103740008F71843189F2863111F41092A5030E94A1
:103750003410809193020E94BA04C6CFD701169606
:103760008C91803108F0FFCEBFCFC801FECE8A9782
:1037700071F780919302811531F08091A50392E059
:1037800089278093A5030E947B0CAECF8C349105D2
:1037900081F38D329240ECCF81E080932F01D6CD22
:1037A00080912F01811169C0C80197558115914001
:1037B00008F0FFC05801F8EFAF22BB24A114B104F8
:1037C00009F0C4CDF801FF2754E0EE0FFF1F5A9512
:1037D000E1F79F01275E3C4F6901D70115968C9157
:1037E000E25EFC4F908180FB90F99083811509F493
:1037F000D8C10E94670890939C0380939B03F601B5
:1038000082818F5F82838091A5039091A103892B90
:1038100083838091A0038483468157816685778561
:10382000C6010E94D707D60115968C9181FF5801D9
:10383000B0929A03A0929903D70115969C91911585
:1038400009F402C610929D039801305723323105C6
:1038500008F008C684E090E00E9491309093ED0358
:103860008093EC03F801E150F047E232F10508F0F3
:10387000E0C1E15EFE4C0C943230380150EE651A26
:1038800071085090A2038091A103582A8091A0034F
:10389000582A88E06816710408F05EC09801277005
:1038A000332781E090E001C0880F2A95EAF73114B0
:1038B00009F44FC0582AD7018D919C910E9442046F
:1038C00021E030E0F90102C0EE0FFF1F8A95E2F718
:1038D000FC87EB8720910F03309110033E832D83EB
:1038E00040911703509118035A87498766E9C62EFD
:1038F00062E0D62EA12CB12C511005C0D601129633
:103900008C9181111BC0F601838190E02B853C8551
:1039100082239323892B91F08085982F97709111A2
:1039200001C087E038E06316710408F066C0311406
:1039300009F45FC086958170811164C09FEFA91A58
:10394000B90AAFE0CA0ED11CB8E0AB16B104A1F6BB
:103950001CC080955822AFCF311038C0809117031A
:10396000909118030817190781F410921803109208
:103970001703109213031092140310921503109260
:103980001603109212031092110380910F0390916D
:103990001003009709F408CFE8E06E16710408F0F0
:1039A000EAC0652D0E940207811103C081E00E94D8
:1039B0007E10F7018581F801E851FC47E730F105F9
:1039C00008F03ACFEF5BFE4C0C94323010931803A2
:1039D000009317030E9480096093130370931403EC
:1039E0008093150390931603109212031092110303
:1039F00062CF82FB882780F99FCF311409F49ECFD4
:103A000080FF9CCFD6018D909C900815190519F464
:103A1000311409F493CFED81FE81EC15FD0509F415
:103A20008DCFD6011D96ED91FC91309721F08081CC
:103A3000811509F483CF652DC6010E940207811507
:103A400009F47CCF81E00815190509F080E0482EC3
:103A500043208114910441F0411006C0E985FA85A4
:103A60008E169F0609F06ACF80E00E947E10D092E9
:103A70001003C0920F0381E080930E038FE08A9DB4
:103A8000F0018B9DF00D1124EA56FD4F8581809346
:103A9000950241100EC08114910459F080819181EA
:103AA0009C0124503109213A310508F049C00E9497
:103AB00058088FE08A9DF0018B9DF00D1124EA5685
:103AC000FD4FC680D780C6019A9581159F4110F49D
:103AD00020EED22299249394C60101978F339E47FA
:103AE00008F0912C8FE08A9DD0018B9DB00D1124A0
:103AF000AA56BD4F1996ED91FC911A97309731F067
:103B00001B966D917C9181E0099598229114A9F002
:103B10008FE08A9DF0018B9DF00D1124EA56FD4F38
:103B2000868197810E94A80380939402C60148E091
:103B30006416710440F40E94A4090E947B0C0AC020
:103B40000E94CA0FB6CF0497813A910548F48C2D94
:103B50000E943F08411409F427CE0E947B0CF6CB4B
:103B60000E947B0C8FE39CE90197F1F700C00000F5
:103B70008C2D8BD8EFCFDC012D913C9102171307D0
:103B800041F4311009C010920E0380E00E947E10B3
:103B90000BCE311409F408CEFC01808585FD04CEDE
:103BA000F4CFF9014485558566857785C9010E9462
:103BB000D707D60115968C9181FF3ECEC6010E9493
:103BC0003D108091990390919A030817190709F005
:103BD00033CE10929A03109299032ECE06E221EE74
:103BE00041EE6AE17CE7B5D9B1CB07E225EE45EEBF
:103BF0006BE17CE7F8CF06E221EE40EE68E17CE77E
:103C0000F2CF07E225EE44EE69E17CE7ECCF06E275
:103C100021EE42EE6CE17CE7E6CF07E225EE46EED0
:103C20006DE17CE7E0CF08E221E045EE6EE17CE764
:103C3000DACF8091EC0381608093EC036091EC0318
:103C40007091ED0384E090E00E94BF300E94CF0CA1
:103C50007DCB8091ED0388608093ED03EFCF809161
:103C6000EC038260E9CF8091EC038460E5CF809122
:103C7000EC038860E1CF8091ED038160EDCF80910E
:103C8000ED038260E9CF8091EC038061D5CF809114
:103C9000EC038062D1CF8091EC038064CDCF0E9491
:103CA000CF0C8091EC038068C7CF8091EC038C60CF
:103CB000C3CF8091ED038360CFCF8091EC038E7FE3
:103CC000BBCF8091ED03877FC7CF8091EC038D7FC1
:103CD000B3CF8091EC038B7FAFCF8091EC03877FD4
:103CE000ABCF8091ED038E7FB7CF8091ED038D7FB9
:103CF000B3CF8091EC038F7E9FCF8091EC038F7DBB
:103D00009BCF8091EC038F7B97CF0E94CF0C80914B
:103D1000EC038F7791CF8091EC03837F8DCF8091DF
:103D2000ED038C7F99CF8091EC03992782FF9395C7
:103D300090FB82F990FB83F97FCF8091ED03982F60
:103D4000909590FB80F990FB81F986CF9091EC03E0
:103D5000892F8F7B96FF80646FCF0E94CF0C90914C
:103D6000EC03892F97FB87F9805866CF61E08EE0DE
:103D700090E00E94A53062CF60E0F9CF9091EC0313
:103D8000892F8F7E94FF806157CF9091EC03892F0C
:103D90008E7F90FF816050CF9091ED03892F877FB8
:103DA00093FF886059CF89E26FC389E258C3073710
:103DB000BCE71B0779F00837ECE71E07A1F0980174
:103DC000205E32452032310598F4911111C0802FC8
:103DD0008F7192CA81E0911541F00E94F40343E093
:103DE00062E081E09CCA82E0F6CF0E94FE03F7CF3A
:103DF00040919F038091A403282F30E020953095B7
:103E000070E024233723232B19F0482340939F038A
:103E10000B37FCE71F0741F4911509F497CA0E947C
:103E2000DB030E94230792CA003422E5120708F040
:103E300055C0003232E5130708F057C0011540E5C0
:103E4000140750F5011550E4150708F064C09115EA
:103E500009F47AC00A35BCE71B0709F4DDC008F095
:103E6000C2C00130FCE71F0709F4D4C003302CE7BF
:103E7000120709F4C9C001151C4709F065C00E946A
:103E8000CF0C8FEF94E3ACE081509040A040E1F77D
:103E900000C000000E94E50998013055211532400C
:103EA000B0F6980145E0369527954A95E1F7822FBF
:103EB0008F7020919F0330E041E050E0082E02C057
:103EC000440F551F0A94E2F724233523232B09F4CA
:103ED000BECF9111A6CF1092A1033FCE9801205CD6
:103EE00032452032310508F0B2CF802F8F712091FA
:103EF0009F0330E041E050E0082E02C0440F551F00
:103F00000A94E2F724233523232B09F4A0CF91153B
:103F100009F41CCA86CFD70116968C91803108F01F
:103F200096CF911111C0212F2F7081E090E002C037
:103F3000880F991F2A95E2F720919F0330E0822392
:103F40009323892B09F002CAD70115968C911597F6
:103F5000CD90DC90811509F463C0C6010E947513F1
:103F6000182F682FC6010E940C04B601812F0E94F1
:103F70005A130E94C6058C01F701B580A680A29451
:103F80002FE0A2228091A6038770811501F1CB2C2E
:103F9000B114F1F0812F807F803461F080E2800FD6
:103FA0008830A8F0812F807E803221F4023078F0B2
:103FB000A11469F08091ED0382FF09C082E00E94A4
:103FC0009F048091A6038770CC24C3948111C12CD7
:103FD000E12FE295EF70103C08F082C0F0E0E85B62
:103FE000FE4C0C9432300B354CE71407B9F080913D
:103FF000ED03002482FF0394802D0C351C4709F04B
:10400000A3CF0E94650CA0CF6FEF7FEF80E090E020
:104010000E94BF300E94F20C81E0F3CF80E0F1CF2C
:10402000C6010E944204182FA0CFF12FFF70DF2E8F
:10403000103118F0D29490EFD922B114A9F0D11414
:1040400059F080E2800F883010F0011107C08D2DEB
:104050000E94BA040E947B0C802F40C08091A5036F
:104060008D298093A503F6CF802F0E94CA0FD1140B
:10407000B9F180E2800F883010F0011104C08D2D5D
:104080000E94C00406C0D0948091A5038D21809326
:10409000A5030E947B0C24C0212F2F70D22E107FED
:1040A000103219F0D29480EFD822011549F0013076
:1040B00009F482C0B11409F48EC0A114A1F1CCCFCF
:1040C0008091ED0382FD2BC0B11419F1D11429F0B8
:1040D0008D2D0E94BA040E947B0C80E00E94451640
:1040E000C11409F4D8C08091A60380FDD4C0D701C3
:1040F00015961C928695869586950E94F403C701B5
:1041000033D88091A6038695869586950E94FE03F6
:10411000C2C080E00E94CA0FD11411F3B0CFB11415
:1041200069F1A11004C08D2D0E941510D9CF31E086
:10413000A31210C01091A0038D2D8123D81681F2F7
:104140000E9467089093AA038093A9031D291093E6
:10415000A003C6CF45E0A412C3CF8D2D0E94151039
:104160008D2D0E9487088091A2039D2D9823D9163A
:1041700009F4B6CF8D298093A203B2CFA11012C04B
:104180008D2D0E941B108D2D0E9487088091A20307
:104190009D2D9823911509F4A3CFD094D822D092C5
:1041A000A2039ECF51E0A5129BCF8091A1038D2148
:1041B000811509F495CFE4CFB11429F086E0A81653
:1041C00008F08ECFB0CF95E0A91608F089CF8D2DDD
:1041D0000E941B1085CFA114D1F3093349F4AFEF2E
:1041E000B7EEE3E0A150B040E040E1F700C00000CE
:1041F000802F0E94CA0F74CF812F86958695837079
:10420000811561F0813009F06BCFC8019370B11056
:1042100002C080E090E00E94170862CFC80193704E
:10422000B11002C080E090E00E94EF0759CF6B2DE3
:10423000802F0E94C50854CF812F8370811138C010
:10424000B11027C0402F429546954770440F440F48
:10425000802F8F70042E01C0880F0A94EAF7202F58
:10426000207104FF07C02FE030E001C0220F4A9503
:10427000EAF720951695169513701230A1F01330B9
:1042800081F03091A303113059F0822B83230E94D7
:10429000EE030E94DC0760E0C7010E949F1366C81E
:1042A000832B822BF4CF822B9091A3038927EFCF0E
:1042B000B11451F110FFEDCF402F42954695477054
:1042C000440F440F802F8F70042E01C0880F0A9472
:1042D000EAF7202F207104FF07C02FE030E001C073
:1042E000220F4A95EAF7209516951695137012300D
:1042F00089F0133069F03091A403113041F0822B22
:1043000083230E94F103C5CF8230B0F6C2CF832B46
:10431000822BF7CF822B9091A4038927F2CF1F70B5
:10432000B11439F0812F0E94F403802F0E941510E0
:10433000B0CF802F0E941B10812F0E94FE03A9CFB7
:10434000023F71F170F4003FC9F0013F91F0B114E8
:1043500009F465C0A11409F45FC0802F0E944516BE
:1043600098CF033F21F1043F91F78091ED0382FD47
:104370002AC0812F8F71B11401F316C0B11469F0F6
:10438000F5E0AF1608F085CF1F7181E090E0012EB7
:1043900001C0880F0A94EAF7BECF26E0A216F2CF3A
:1043A000812F8F71B110C9CF0E94F40372CF80E0CA
:1043B000B11409F4A6CF1F7181E0012E01C0880F4E
:1043C0000A94EAF79ECFB114C1F08091A6038770DA
:1043D000843049F41092A6031092A8031092A70308
:1043E000812F8F71AACF35E063E0A31608F051CF7B
:1043F000812F8F710E9473084CCF45E0A41640F0C6
:104400001092A6031092A8031092A70364E0F0CFC5
:1044100081E00E949F043DCF812F8F71C5CFA114F1
:10442000F9F2093349F45FEF87EE93E05150804091
:104430009040E1F700C00000802F0E94CA0F29CFF2
:104440000337BCE71B071FC90631ECE71E0709F05D
:10445000AECC80919E03811509F4A7CC85E30E9420
:1044600058087BCB0631FCE71F0709F0A0CC8091F0
:10447000A1038A7A91E0811101C090E090939E039C
:10448000811509F490CC85E30E943F0866CBA0E03B
:10449000B0E0EDE4F2E20C94F32F8091EB03803175
:1044A00008F049C08091EA03811509F444C0C09125
:1044B000AC0387E0D82E8091AB038C17E1F1EC2E92
:1044C000F12CDC9EE0011124FE01E355FC4F8481B8
:1044D0008115B1F191818091E603981331C09081EB
:1044E0008091E50398132CC08581811129C0028138
:1044F00013818091E7039091E803081B190B60E09A
:1045000085EE93E00E949F130E9427150817190754
:10451000B8F48091EB038F7080618093EB03CD54EE
:10452000DC4F88818F708061888385EE93E00E94E4
:10453000B4180E949504CDB7DEB7E7E00C940F30B5
:10454000E7012196C770B7CFADE0B0E0EAEAF2E24A
:104550000C94EB2F8C0186E0F801DE011896019097
:104560000D928A95E1F7F801F580E48085EE882EBA
:1045700083E0982E8091E903811117C0E11491F036
:10458000F11409F455C1C8010E94CA13811509F438
:104590004FC187E0F801A5EEB3E001900D928A9536
:1045A000E1F775DFFF24F39461C0A280B380D0905F
:1045B000EA038091E7039091E8033501681A790ACC
:1045C000D11409F4F0C0C080518060E085EE93E022
:1045D0000E949F130E9427156816790608F09EC056
:1045E000E11401F38091E603F8019181E090EB037F
:1045F000F0E1EF1608F05BC0981317C09091E50347
:10460000F8018081981311C0F1104BC08E2D8F706E
:1046100080618093EB0385EE93E00E94B418809153
:10462000EB03F8018683F12C21C0F1103AC040E081
:10463000652D8C2D0E94700B40E0652D8C2D0E9405
:10464000700BF82E8111EFCF888599850E94BD13DC
:10465000292F22952F70903470F49F702230A0F093
:104660009115B1F0F8019681903190F48F2D2D962F
:10467000EFE00C9407302A5F2F70223068F0C801F9
:104680000E94B418FD2CF2CF911511F0811571F331
:10469000805E883058F3F3CF803F40F3815F8330F2
:1046A000F9CF8091EB0381608093EB03BCCF98132B
:1046B00015C09091E503F801808198130FC0F110A7
:1046C0000DC0E682C8010E94B41887E0F801A5EE8B
:1046D000B3E001900D928A95E1F764CFC8010E9482
:1046E000CA13811509F4A4C0F11409F4A1C0809182
:1046F000EB03803208F44DCF8091E5039091E603FF
:104700009A838983BC82AB828091E9038D831E8268
:10471000EF82CE0101960E94B4183BCFD090EB03FC
:10472000F0E1DF1650F485EE93E00E94B41887E0C4
:10473000F40111928A95E9F776CFE11409F432CFAA
:104740009091E603F8018181981311C09091E503DF
:10475000808198130CC0F1100AC0D682C8010E9453
:10476000B41887E0F40111928A95E9F71BCFC801CC
:104770000E94CA13811509F45BC0F11409F458C0F2
:104780008091EB03803208F404CF8091E50390918F
:10479000E6039A838983BC82AB828091E9038D838F
:1047A0001E82DF82B6CF60E085EE93E00E949F1309
:1047B0000E9427156816790608F0B9CFE11409F4AC
:1047C000F1CEF114A9F19091E603F80181819813DB
:1047D00025C09091E5038081981320C08091E70364
:1047E0009091E803A81AB90AF8ECAF16B10408F0E2
:1047F0006CCF8091EB0380FD68CF803108F465CFEA
:10480000F8018683982F907F903F09F45BCF982F13
:10481000907F905F8F70892B868354CFC8010E9450
:10482000CA138111B6CE8091EB0381608093EB03B4
:10483000C8010E94B418B6CEABE1B0E0E2E2F4E207
:104840000C94F62F4E8B5F8B688F798F8A8F192F80
:104850009B8F91111092A5031D8A86E0FE0176962A
:10486000DE011F9601900D928A95E1F70A8D8091E5
:10487000ED0382FF1FC00E9467082091A7033091BB
:10488000A803821B930B8838934138F08091A603CC
:1048900082FD03C082E00E949F040E94670820916D
:1048A000A9033091AA03821B930B8838934110F01F
:1048B0000E94C804011561F00B8B1C8B61E0CE01D6
:1048C0000F960E949F1361E0CE010F960E949F13E6
:1048D0000B8B1C8B87E0FE013F96DE011896019042
:1048E0000D928A95E1F7CE0108962EDE811110C057
:1048F0002091AB033091AC0387E0FE013896DE01D6
:10490000119601900D928A95E1F78C8581110BC06B
:1049100017E08091AC039091AB0389132BC06B9689
:10492000E4E00C941230822F90E001968770992772
:104930003817190671F40E94CF0C1092AB03109235
:10494000AC0387E0E5EEF3E0DF011D928A95E9F71D
:10495000DFCF97E0929FD0011124A355BC4FFE01F9
:10496000319601900D929A95E1F78093AB030E94E6
:104970009504CECF189FC001112483559C4FE4DDD0
:10498000811569F28091AC0390E0019687709927B8
:104990008093AC03BECFA6E0B0E0E1EDF4E20C946E
:1049A000F62F0E9467088C01809155029091560263
:1049B0008017910771F019821A820E946708BC0162
:1049C00049815A8180E090E037DF109356020093CE
:1049D00055022696E4E00C941230A6E0B0E0E3EF36
:1049E000F4E20C94F82F90935202809351028115B7
:1049F00020E2920730F40E947E172696E2E00C94A3
:104A0000143080EF89838A830E9467088160BC012B
:104A100049815A8181E091E00FDFEFCFA6E0B0E05D
:104A2000E4E1F5E20C94F62F8C019093520280930E
:104A30005102011580E21807B0F4802F0E94CA0FBE
:104A4000C801805E9109089728F06AE270E10115BB
:104A5000110511F46BE170E1C8010E94D2032696A2
:104A6000E4E00C94123080EF89838A830E94670807
:104A70008160BC0149815A8181E090E0DDDEEFCFA9
:104A8000CF93DF93D82FC92FA8DF8D2F9C2FC6DFA0
:104A9000DF91CF9108950F931F93CF93DF938C01F4
:104AA000862F66E872E00E941215892B91F4C0915E
:104AB0008602D0918702209761F0F80182818330CD
:104AC00039F4CE01DDDFCE01DBDFCE01D9DF01C05D
:104AD000E0F7DF91CF911F910F9108950F931F93EE
:104AE000CF93DF938C01EB0166E872E08C2F0E947C
:104AF0001215892B09F057C0FE01FF27D801129625
:104B00008C911297EB50FE4F8130A9F415968C9141
:104B100082FD4EC080FF4CC082E08083809188027D
:104B2000909189020097B9F4809186029091870252
:104B30000097C9F110C08230A1F515968C9182FDC5
:104B400026C080FD0AC083E0808380918A02909114
:104B50008B020097F1F041DF26C084E080838091D2
:104B60008C0290918D020097B1F78091860290910E
:104B70008702009701F184DF809188029091890279
:104B8000009749F78091860290918702E4CF85E0F3
:104B900080838091860290918702009721F070DFD8
:104BA000F1CF86E08083DF91CF911F910F9108951F
:104BB00081E08083B9CF8091880290918902B8CF3B
:104BC0000F931F93CF93DF938C01EB0166E872E0A4
:104BD0008C2F0E941215892B71F4DD27CB50DE4FEC
:104BE0008881F801128218828330E9F048F481301C
:104BF00059F0823081F0DF91CF911F910F9108958C
:104C00008430B1F08530B9F78091860290918702A7
:104C1000009789F306C080918802909189020097DD
:104C200099F3FCDEE8CF80918A0290918B02F7CF56
:104C300080918C0290918D02009799F720918602C5
:104C40003091870280918802909189022115310567
:104C5000F9F2009731F7C901E4CFCDB7DEB7AC97D1
:104C60000FB6F894DEBF0FBECDBF85B7806885BF95
:104C700085B7806885BF84B7877F84BF0FB6F894F7
:104C8000A895809160008861809360001092600018
:104C90000FBE80E890E00FB6F89480936100909387
:104CA00061000FBE81E08093030182EC96E0909357
:104CB000C3018093C2010E94EA060E9493140E94DD
:104CC000A00A0E94160B8091E20084608093E200AB
:104CD000789480913302811599F08091E9001091C8
:104CE000EC008F70179511271795182B1092E9007B
:104CF0008091E80083FD0E94070D1F701093E9006A
:104D000082E084BD93E095BD9AEF97BD80936E00DD
:104D100010924D0210924E0210924F0210925002C9
:104D20000E940514811102C00E947C158091D80058
:104D300080618093D8002AE12A95F1F700C0809124
:104D4000D900182F117080FD04C00E94A00A109293
:104D5000330210934B0210934C0210930401111173
:104D6000E4D7809104018091040190E0811101C099
:104D700095E09093080285E0891B8093070208E480
:104D800011E0D8018D918D018F3F11F00E94C40672
:104D9000B1E00D341B07A9F70DE411E0F801819192
:104DA0008F018F3F11F00E94C406F1E003351F0709
:104DB000A9F78AE0E7E2F2E0DF01282F1D922A95A9
:104DC000E9F7EDEFF1E0DF011D928A95E9F780E068
:104DD00090E00E949130833E9E4F21F40E94051482
:104DE000811102C00E94A11582E090E00E948930EA
:104DF00080930B0284E090E00E9491309093ED0349
:104E00008093EC030E94D910EFEFF6E721E0E15028
:104E1000F0402040E1F700C000000E94D9108091CE
:104E2000270280FF08C06FEF7FEF80E090E00E94D4
:104E3000BF300E94E50983E090E00E9489300E9423
:104E4000EE0380914B02811101C072D785E091E0A1
:104E5000909358028093570280913302853049F431
:104E600080913302853009F451C00E94CF0C0E941A
:104E7000DC070E94D9100CE012E057E2E52E52E068
:104E8000F52ED701F80191918D9126E132E02E1790
:104E90003F0709F470C09817B1F370904B02D12C02
:104EA00088248394D701CD907D01F80191908F01E2
:104EB0009C1429F19C24B12CAA24A394892D8A2125
:104EC0008115B1F07114A1F0B982DA820E946708ED
:104ED0009C838B838D8291E08C2D8A21811101C06E
:104EE00090E09E8349815A816B817C818D81A4DC15
:104EF000B394AA0CF6E0BF12E1CFF801C292D394AA
:104F00002AE0D212CFCF0E948C0938C080913302A0
:104F1000843021F11092090288E190E0A0E40FB6FC
:104F2000F894A895809360000FBEA093600083B7AB
:104F3000817F846083BF83B7816083BF78948895C5
:104F400083B78E7F83BF0FB6F894A89580916000D9
:104F5000886180936000109260000FBE0E94D9109B
:104F6000E7E2F2E081918111F2C421E332E02E17F1
:104F70003F07C1F775CF981390CF0DDD80914B029D
:104F8000811509F478C000911103109112030115E5
:104F9000110591F1C0901A02D0901B02E0901C0202
:104FA000F0901D020E9480096C197D098E099F09ED
:104FB000C0901602D0901702E0901802F0901902EB
:104FC0006C157D058E059F05B8F0C8010E947E17FF
:104FD000109211031092120310921A0210921B02E7
:104FE00010921C0210921D021092160210921702CB
:104FF0001092180210921902E0909903F0909A030F
:10500000E114F10439F1C0909B03D0909C030E94FD
:1050100067088C010C191D09C7010E94271580170C
:105020009107C0F42091990330919A03C9019927FF
:10503000287F3327232B09F009C144E0880F991FEB
:105040004A95E1F7875E9C4FDC0115962C9122FF73
:105050000E94591080919002811569F00E946708A2
:105060002091910230919202821B930B8F3F9F47B8
:1050700010F40E94341086E0E0E8F2E0DE011196C0
:1050800001900D928A95E1F7B0908102D090820252
:1050900010918302C09084020091850210928202D6
:1050A000109283021092840210928502812F8D2922
:1050B0008115A1F0E0902002F09021020E94670883
:1050C0009C012E193F0990917E02911509F4C1C0EF
:1050D00080912D018217130608F4C9C08C2D802BF6
:1050E000811509F441C0E0901E02F0901F020E9459
:1050F00067089C012E193F0990917D02911509F4D2
:1051000021C42135310580F19F3F19F09F5F9093B5
:105110007D02C11459F00E949E0791E01C140CF00E
:105120009FEF899F802D112480938402011559F0EF
:105130000E949E0791E010160CF09FEF899F802D32
:1051400011248093850280918402811569F0F0908A
:105150008502F11449F00E944A07809384028F2D42
:105160000E944A0780938502809181028B1119C0A9
:1051700080918202811511F08D1113C0209183025C
:10518000211511F021130DC090918502911511F098
:10519000901307C030918402311103C0822B892BF8
:1051A00081110E949C0886E0FE013196A0E8B2E0E1
:1051B00001900D928A95E1F70E94DC0790912202FE
:1051C000891721F0809322020E9480098091330286
:1051D000843009F041CE83E08093E9008091E800BB
:1051E00082FF3ACE8091E80090E085FF0CC00E94DB
:1051F0006F0A30E2E32EF12C8E010F5F1F4F8115F5
:1052000009F46FC091E08091E8008B778093E8000B
:10521000911509F421CE0091530210915402E981B5
:105220000115110509F46BC0EE3F09F08BC08A81AE
:10523000833020F08550833008F084C0EA81EE305E
:1052400008F080C0F0E0EC5AFE4C0CC780E090E023
:10525000FBCE40912E01EAE04E9FA001112442179F
:10526000530708F03BCF9F5F90937E0202C09F3FA1
:10527000D1F7D11459F00E94580791E01D140CF099
:105280009FEF899F802D112480938202111559F080
:105290000E94580791E011160CF09FEF899F802D16
:1052A00011248093830280918202811509F416CF24
:1052B000F0908302F11409F411CF0E944A07809301
:1052C00082028F2D0E944A078093830207CF80912C
:1052D000F100D8018D938D01B1E0EB1AF10809F4CA
:1052E00091CF8091E80085FDF2CF8091E8008B7727
:1052F0008093E8000E946F0A811599F383CFE4310F
:1053000048F4E11551F0E150E33138F4F0E0EE59A2
:10531000FE4CA8C6EE3F09F491CF8FEF898312C0EF
:105320001A8289E08B830EC08A81823081F08330BB
:10533000B1F0813091F70E9480099AD66B837C830B
:105340008D839E83CE0101960E94BF0A85CD88E29F
:1053500090E0DFD61B821C821D828E83F3CF80916A
:10536000310290913202892B69F38AE0E7E2F2E0A0
:10537000DE01139601900D928A95E1F7E3CF8A81C1
:10538000823059F66B817C818D819E8171D688E255
:1053900090E0DBD6D7CF4C816B818A810E942B13A2
:1053A0009827892798279E838D83CCCF2D813E8196
:1053B0003227232732274C816B818A810E943E0C41
:1053C000C1CF0E941E14BECF80E18A83BBCF1A8258
:1053D00087E6A8CF8C818D3108F0B4CF8A809B807E
:1053E000982489249824A12CB12CFE0131967F01A8
:1053F0008F01080F111DE016F10609F4A3CF80E01C
:10540000F7E68F169104A104B10420F4C401875675
:105410009C4F7FD6D70114968C93BFEFEB1AFB0AF3
:10542000EFEF8E1A9E0AAE0ABE0AE5CF80913102D6
:1054300090913202892B09F485CF8C818D3108F04F
:1054400081CF882E912CA12CB12CCA80DB80DC244A
:10545000CD24DC24E12CF12C8E010F5F1F4F412C59
:10546000512C3201481459046A047B0408F06ACFB5
:10547000F7E6CF16D104E104F10438F4D80114960C
:105480006C91C60187569C4F60D6BFEF4B1A5B0AE2
:105490006B0A7B0AEFEFCE1ADE0AEE0AFE0A0F5FF6
:1054A0001F4FE0CF0E9442154DCF86E08ECF8C81FA
:1054B0008D3108F047CF882E912CA12CB12CCA80B9
:1054C000DB80DC24CD24DC24E12CF12C412C512C7C
:1054D00032018E010B5F1F4F481459046A047B048C
:1054E00008F030CF80E0F0EDCF16F2E0DF06E10407
:1054F000F10418F4C60189960CD6D8018D938D015C
:10550000BFEF4B1A5B0A6B0A7B0AEFEFCE1ADE0A7B
:10551000EE0AFE0AE1CF2C81022F10E02D3108F0B7
:1055200011CF8A819B819827892798272C01612C8C
:10553000712C803DF2E09F0708F004CF822E912C61
:10554000A12CB12C40ED52E060E070E04419550907
:1055500066097709421751056105710508F4F2CE15
:105560002091310230913202232B09F03EC01C0100
:1055700029E2220E311C80FBEE24FF24E0F880FF9C
:105580000BC08896C6D59D818927982789278115C4
:105590009C4711F48FEF8D83D501C401840D951DB7
:1055A000A61DB71D80FF19C0680181E0C81AD10887
:1055B000DE011596AC0DBD1DBCA7ABA7C101800FC8
:1055C000911FA7D5EBA5FCA5908181159C4721F4DF
:1055D0008FEFABA5BCA58C938601FE013196EE0D35
:1055E000FF1D2FEFE016F10638F08E010F5F1F4F01
:1055F000C12CD12C760125C09481858181159C47D1
:1056000011F42483258332E0E30EF11C3296EACFB5
:1056100080ED481682E058066104710430F4D80128
:1056200014966C91C201899690D5BFEFCB1ADB0A14
:10563000EB0AFB0AEFEF4E1A5E0A6E0A7E0A0F5F54
:105640001F4FC814D904EA04FB0410F37BCE8091E9
:10565000310290913202892B09F474CECE01019669
:105660000E94BF0AFFEF21EE34E0F15020403040AD
:10567000E1F700C00000DDCB88E0E0E3F1E0DE010F
:10568000919601900D928A95E1F7FE0132968FE195
:10569000DF011D928A95E9F786E0898388E07F968D
:1056A000DE01159667CE88E4898381E08A831B82B8
:1056B0001C8248CE8B819C81092E000CAA0BBB0B4F
:1056C00025E0880F991FAA1FBB1F2A95D1F7AC01AF
:1056D000BD01405E5F4F6F4F7F4F481759076A0704
:1056E0007B0708F42FCE8834E1E09E07A105B105C1
:1056F00008F028CE4934F1E05F076105710520F01C
:1057000048E451E060E070E0481B590BBC01645371
:105710007A4FCE010196C7D415CE4AE150E06FEF23
:1057200070E0CE010796DED48091310289830A832E
:105730001B821C821D8281E010CE81E090E090935C
:1057400054028093530282E390E090932602809368
:1057500025020E9467089093240280932302F2CDD1
:105760000115110571F1D0902702E0902302F0900D
:1057700024020E9467088E199F098536910540F121
:10578000D1FE26C0D0FE24C00E9467089093240258
:105790008093230280912502909126020197909395
:1057A000260280932502892B61F4109254021092F4
:1057B000530281E090E0909332028093310200E046
:1057C00010E08091310289830A8380912502AACD5D
:1057D00082E390E09093260280932502F2CF10920C
:1057E000320210923102AECD40E250E06FEF70E035
:1057F000CE01019677D4A6CD8B81823009F450C0BA
:1058000078F4811136C0FE0132968EE1DF011D92DF
:105810008A95E9F788E089838B8383E088A392CD1A
:10582000853009F472C0863009F08CCD1C818AE085
:10583000FE013596DE01919601900D928A95E1F771
:105840008BA19CA10E94DD069CA38BA38FEF183037
:1058500060F4FAE01F9FB0011124675B7C4F4AE0BF
:1058600050E0CE0181968FD480E089830E9493140A
:1058700069CD8C819AE0F92E8E010F5D1F4FF801E2
:105880002F2D11922A95E9F7B8010E9412158983EC
:10589000F801DE01129601900D92FA94E1F752CDD3
:1058A0001C818AE0FE013596DE01919601900D92F1
:1058B0008A95E1F789A19AA10E94DD069AA389A39E
:1058C0008BA19CA10E94DD069CA38BA38DA19EA110
:1058D0000E94DD069EA38DA38FA198A50E94DD06E0
:1058E00098A78FA38FEF183060F43AE0139FB001B0
:1058F000112467507D4F4AE050E0CE01819643D499
:1059000080E089830E94EA061DCD2C816AE0CE01E9
:105910008196DC01E62F1D92EA95E9F7283080F4A4
:10592000629FB0011124675B7C4F4AE050E0E1D3F5
:1059300080E089838AE0FE01B196DE0112961ACDDD
:105940008FEFF7CF2B30310508F0E0CB0DCC8091F5
:105950000A02811509F484CA30E139BD82E189BDAA
:1059600009B400FEFDCF8091D8008F7D8093D800D0
:105970008091E00082608093E0008091E00081FDF2
:10598000FCCF0E94CF0C6CCA1F921FB61F9211242D
:105990008F939F93AF93BF9380910902811113C09E
:1059A0008091EC019091ED01A091EE01B091EF0199
:1059B0004196A11DB11D8093EC019093ED01A09340
:1059C000EE01B093EF01BF91AF919F918F911F9026
:1059D0001FBE1F90189578941F921FB61F92112416
:1059E0008F939F93AF93BF938091EC019091ED01C2
:1059F000A091EE01B091EF010196A11DB11D809320
:105A0000EC019093ED01A093EE01B093EF01BF91F3
:105A1000AF919F918F911F901FBE1F9018951F925D
:105A20000F920FB60F9211242F933F934F935F93D2
:105A30006F937F938F939F93AF93BF93EF93FF9356
:105A40008091E10082FF09C08091E20082FF05C0E1
:105A50008091E1008B7F8093E1008091DA0080FFEC
:105A600024C08091D80080FF20C08091DA008E7F12
:105A70008093DA008091D90080FFA9C080E189BDC0
:105A800082E189BD09B400FEFDCF81E0809333023D
:105A90008091DB01811109C00E94A00A0E94160BAF
:105AA0008091E20084608093E2008091E10080FFB9
:105AB0001AC08091E20080FF16C08091E2008E7FC4
:105AC0008093E2008091E20080618093E200809107
:105AD000D80080628093D80019BC85E0809333029F
:105AE00083E0809303018091E10084FF2FC08091C7
:105AF000E20084FF2BC080E189BD82E189BD09B449
:105B000000FEFDCF8091D8008F7D8093D8008091DA
:105B1000E1008F7E8093E1008091E2008F7E809390
:105B2000E2008091E20081608093E2008091DA01DE
:105B3000811509F452C084E08093330280913302CE
:105B4000843009F052C082E0809303018091E1002B
:105B500083FF2CC08091E20083FF28C08091E10088
:105B6000877F8093E10082E0809333021092DA0114
:105B70008091E1008E7F8093E1008091E2008E7F32
:105B80008093E2008091E20080618093E20042E035
:105B900060E080E00E94E60A8091F00088608093D7
:105BA000F00081E08093030180930201FF91EF9167
:105BB000BF91AF919F918F917F916F915F914F9125
:105BC0003F912F910F900FBE0F901F90189519BC09
:105BD000109233021092DB0168CF8091E30087FFBF
:105BE00002C083E0A9CF81E0A7CF81E0ADCF1F92B3
:105BF0000F920FB60F921124EF92FF920F931F9303
:105C00002F933F934F935F936F937F938F939F93C4
:105C1000AF93BF93CF93EF93FF9309EE10E0F8019A
:105C20008081C091EC008F70C795CC27C795C82B99
:105C3000108280EFE82EF12CF7018081877F80832E
:105C400078940E94070DF8011082F7018081886026
:105C50008083CF70F801C083FF91EF91CF91BF9106
:105C6000AF919F918F917F916F915F914F913F91F4
:105C70002F911F910F91FF90EF900F900FBE0F90FB
:105C80001F9018958EE1489B02C08A95E1F7489BCA
:105C9000FECF0895589880E28A95F1F7589A0895B2
:105CA000FC012BE02A95F1F728E090E080E031E05C
:105CB00040E14A95F1F7880F489B02C08160932725
:105CC00042E04A95F1F7000040E14A95F1F72A9544
:105CD00079F720E12A95F1F729B132E03A95F1F709
:105CE000000040E14A95F1F7217092272081920F40
:105CF00090830895A1E0B0E0EFE7FEE275C119825C
:105D00008C017C01E60EF11CBDDFCE010196C8DFDF
:105D1000F80181938F01EE15FF05B1F781E09981BC
:105D2000911180E02196E6E07BC1509A589A08953F
:105D30005098589AE89AE9E6F0E080818C7F808359
:105D400008956150770B91E001C0990F6A95EAF7C9
:105D5000692F90E021E0611108C0911599F0589ADF
:105D600080E28A95F1F758980895362F3823311537
:105D700039F0589A922730E23A95F1F76695EBCFD1
:105D80005898F9CF5898ECCFFF920F931F93CF9369
:105D9000DF93EC018C01060F111DF9907BDF68E0A9
:105DA0008F2DCFDFC017D107C1F7CDB7DEB7E5E044
:105DB00038C11F920F920FB60F9211240F931F93A9
:105DC0002F933F934F935F936F937F938F939F9303
:105DD000AF93BF93EF93FF93CF93DF930F92CDB722
:105DE000DEB719824FDFCE0101965ADF082F0695E4
:105DF00006950695982F92959570202F2570920FF5
:105E0000292F237096959695920F982797708981E0
:105E1000892B811509F058C0043008F055C080E185
:105E20008A95F1F7589A509A82E08A95F1F700C066
:105E3000589888E0089F80011124D801AF5EBE4FBA
:105E40001696ED91FC9117973097A9F06091530148
:105E50007091540114962D913C911597260F371F80
:105E600011968D919C911297680F791F13964C9102
:105E700013978C910995F801EF5EFE4F63816115D0
:105E800049F0209153013091540184819581820F12
:105E9000931F7ADFFFDE80E18A95F1F758985098DA
:105EA000589A80E18A95F1F7F801EF5EFE4F608124
:105EB000611549F020915301309154018181928103
:105EC000820F931F17DFDEDE0F90DF91CF91FF91DE
:105ED000EF91BF91AF919F918F917F916F915F9162
:105EE0004F913F912F911F910F910F900FBE0F90E7
:105EF0001F9018950F931F93CF93DF938C010497F6
:105F00000CF05EC0F894509A589885E08A95F1F7A5
:105F10000000C02FC695C570802F8570C80F8C2FCC
:105F20008370C695C69593E0000F111F9A95E1F70F
:105F3000C80FC8018C2BEC01ADDE00C068E08C2FCF
:105F400000DF90E19A95F1F75098589A489B31C03C
:105F500087E090E048992FC0F801EF5EFE4F638123
:105F6000611559F02091530130915401848195813C
:105F7000820F931FBFDE811501F184DE80E28A95D6
:105F8000F1F75898509A90E19A95F1F7F801EF5E81
:105F9000FE4F6081611549F0209153013091540109
:105FA00081819281820F931FEFDE74DE789481E00D
:105FB00008C000C0CBCF019749F4509A589A789402
:105FC00080E0DF91CF911F910F91089500C0C2CF63
:105FD0002F923F924F925F926F927F928F929F92F9
:105FE000AF92BF92CF92DF92EF92FF920F931F93E7
:105FF000CF93DF93CDB7DEB7CA1BDB0B0FB6F89498
:10600000DEBF0FBECDBF09942A88398848885F84D7
:106010006E847D848C849B84AA84B984C884DF8048
:10602000EE80FD800C811B81AA81B981CE0FD11D2C
:106030000FB6F894DEBF0FBECDBFED01089597FBFC
:10604000072E16F4009406D077FD08D018D007FC70
:1060500005D03EF4909581959F4F08957095619578
:106060007F4F0895EE0FFF1F0590F491E02D0994E6
:106070006927962769277827872778270895AA1BF5
:10608000BB1B51E107C0AA1FBB1FA617B70710F023
:10609000A61BB70B881F991F5A95A9F78095909555
:1060A000BC01CD010895FB01DC0102C005900D92F9
:1060B00041505040D8F70895FB01DC0104C08D9198
:1060C0000190801921F441505040C8F7881B990B6A
:1060D0000895FB01DC0102C001900D924150504037
:1060E000D8F70895DC0101C06D9341505040E0F7AE
:1060F0000895DC01CB01FC01F999FECF06C0F2BD89
:10610000E1BDF89A319600B40D9241505040B8F775
:106110000895F999FECF92BD81BDF89A992780B56F
:106120000895A8E1B0E042E050E0E5CFDC01A40F23
:10613000B51F4150504040F0CB01840F951F2E9168
:1061400005D041505040D8F70895262FF999FECF39
:1061500092BD81BDF89A019700B4021639F01FBABA
:1061600020BD0FB6F894FA9AF99A0FBE08950396D7
:10617000272FECDFEADF252FE9DF242FE7CF019679
:10618000272FE4DFE2CFDC01CB0102C02D9105D047
:1061900041505040D8F70895262FF999FECF1FBAE5
:1061A00092BD81BD20BD0FB6F894FA9AF99A0FBE40
:1061B00001960895F894FFCFD108D608D808DD08D5
:1061C000ED08ED08ED08ED08ED08ED08ED08ED0827
:1061D000DF08E308E608EB08FB0801090509E40D00
:1061E0000A0E100E0A0E100E620E830E100E890F8C
:1061F000960FF715EE150A16EC15E115E115EC15DD
:10620000E115E1152616E1153116E115E115E11547
:10621000E115E115EC15E115E115EC15E115181680
:10622000E115E1154316431643164316431643166C
:10623000431643164316E515E115F715EB155D1EDC
:10624000C51E651E2F1E331E691E371E6D1E791E4C
:10625000431EBE1E471E7D1E4B1E811EA61E4F1EC8
:10626000851EAD1E551E8B1E931E3B1E711E3F1EAE
:10627000751E591E8F1E9D1EB61EBC1E291E611E38
:10628000CC1EFB1D011EEE1DF51D071E0D1E131E4F
:10629000152015204C204C20FC2017217020702048
:1062A0001C218F21A021A0213C2B532B5A2BA2294A
:1062B000A2298D2B9D2BB02BEF2BF42BA229A229E9
:1062C000A229FC2B90299429BF29CB29D629E12981
:1062D0008D298D298D298D29272BE429E729EA2964
:0A62E000162A522A552A572A8B2A43
:1062EA0000000100016408D10BF609E70BEC0BC8AA
:1062FA000B00000001000000000000000501000082
:10630A0000040600000000000028081E0A1401010B
:10631A00BBBBAD3D7081F6410044227B4901270198
:10632A00AC004F02680288029497C63435F6F731FA
:10633A003332363802E200E900EA00B500B600B7A7
:10634A0000CD008301CC008A01920194012102232D
:10635A000224022502260227022A02B300B4006F91
:10636A000070009F01CB019F02A002E200E900EA4F
:10637A0000B500B600B700CD008301CC008A0192B7
:10638A000194012102230224022502260227022A5D
:10639A0002B300B4006F0070009F01CB019F02A0FE
:0263AA000200EF
:00000001FF
